:100000000C947A000C9412020C9497000C949700B4
:100010000C9497000C9497000C9497000C94970004
:100020000C9497000C9497000C9497000C949700F4
:100030000C9497000C9497000C9497000C949700E4
:100040000C9497000C9497000C9497000C949700D4
:100050000C9497000C9497000C9497000C949700C4
:100060000C9497000C9497001201100102000008F4
:10007000C016E10500010102000110035500530004
:1000800042002D0032003300320022037700770057
:1000900077002E0072006500630075007200730027
:1000A00069006F006E002E006A00700004030904EE
:1000B000090243000201008032090400000102022B
:1000C0000100052400100104240202052406000199
:1000D0000524010301070583030800FF090401004B
:1000E000020A00000007050102080000070581025E
:1000F0000800000011241FBECFEFD8E0DEBFCDBF47
:1001000011E0A0E0B1E0EAE6FAE002C005900D924D
:10011000AC30B107D9F722E0ACE0B1E001C01D92EC
:10012000A43EB207E1F70E94BE040C9433050C9480
:1001300000001F93CF93DF93162FEA01288124FF3D
:1001400017C0298138E823272983212FFC01CE01FC
:100150000296DC0131913D9321501216DCF3612FA0
:100160000E940E021C5F1883DF91CF911F910895AA
:100170002AE52883EACF40E251E00C9499004BE451
:1001800051E00C949900CF93DF936091310163505B
:1001900067FD16C080912E01CCE0D0E0C81BD109CC
:1001A000CB5CDE4F80912D01803108F047C0CE013D
:1001B0000E94A10480913101181614F410923101AB
:1001C0008091010184FF2DC0809100018F3F49F192
:1001D000C82F893008F0C8E08C1B80930001809103
:1001E000150198E8892780931501CC2369F0809147
:1001F0000C0187FFC2C06C2F86E191E00E9464046D
:10020000C82F893008F0DDC06C2F86E191E00E9494
:100210000E02CC5FCC3019F08FEF80930001C093B9
:10022000010184E199B1947831F48150D9F71092A9
:10023000320110922C01DF91CF9108958D3209F097
:1002400089C0683009F0B6CF83EC809315018AE548
:100250008093010110920C018881807671F0CE01AB
:100260000E9441048F3FC1F4988197FD8E8190E8F0
:1002700090930C01809300019DCF2A8110921E0162
:100280009981911111C010921F012EE131E082E09D
:100290003093300120932F019F819111EBCF9E81EC
:1002A000981740F7892FE6CF953029F42093320133
:1002B0002EE131E0EDCF9630A1F59B81913059F4DC
:1002C00088E690E09093300180932F0182E190E4E2
:1002D00090930C01C7CF923021F4CE010E942C04E0
:1002E000F6CF9330A1F7211108C08CEA90E09093EB
:1002F000300180932F0184E0EACF213041F48AE875
:1003000090E09093300180932F0182E2E0CF223081
:10031000F1F68AE790E09093300180932F0180E11D
:10032000D6CF983081F0993019F420933401C0CFA2
:100330009A3069F09B3009F0BBCF9BE49093210188
:1003400090934C01B5CF24E331E081E0A1CF2EE1C1
:1003500031E0FBCF80910C0187FF2CCFCE010E94B2
:100360007F048F3F21F48EE18093010123CF882306
:1003700009F420CF109200011DCF40912F01509120
:10038000300186FF15C0A6E1B1E0FA019C2F8491EF
:100390008D9331969150D9F72FEF2C0F30E02F5FCE
:1003A0003F4F240F351F3093300120932F012CCF66
:1003B000DA01E6E1F1E09C2F8D9181939150E1F714
:1003C000EBCF8FEF80930001CEE129CFE9E6F0E09B
:1003D000808182608083E89AA0E2B1E08BE411968C
:1003E0008C931197EBE4F1E081838AE58C93808311
:1003F0000895A82FB92F80E090E041E050EA609581
:1004000030E009C02D9182279795879510F08427B9
:100410009527305EC8F36F5FA8F30895EADF8D93E8
:100420009D930895CF93CFB7CF93DF93C3954F9B01
:10043000E9F74F9B0BC04F9B09C04F9B07C04F9BD9
:1004400005C04F9B03C04F9B01C08EC06F93C091EE
:100450002E01DD27CB5CDE4F2F9365E54F9B03C05C
:100460002F916F91E6CF0F931F934F9320E040E1C0
:100470005F9309B1047807FB27F93F9350E03BE015
:1004800039C0147840642F77012F5F5F1EC0406829
:1004900019B114782F7752501FC0406409B12F77DB
:1004A0000478D1F15F5F00C023C0406219B12F779B
:1004B000147891F15F5F00C025C004781027515077
:1004C00012F45D5F0000115027952C3F19B1C8F65A
:1004D00014780127015027952C3FC8F642274993ED
:1004E00009B1047810274F73115027952C3FA8F6B7
:1004F0004695469519B1147879F001270150279552
:100500002C3F98F66B5A60F3315009B1B0F600C039
:1005100011E01CBB00271CC03B503195C31BD040D1
:1005200011E01CBB0881033C21F10B3411F1209137
:100530002C011981110F1213EDCF4A81441F093686
:1005400069F10D3211F0013E29F74F7009F0042FC7
:10055000009333013F915F914F911F910F912F9124
:100560006F91CCB3C0FD62CFDF91CF91CFBFCF9160
:10057000189520913301222369F310913101112341
:10058000E9F53430EAF13093310120932D011091D7
:100590002E013BE0311B30932E0132C0009131011E
:1005A000013064F50AE54F7049F43091010134FDE2
:1005B00028C000930101C5E1D1E027C0433049F0D4
:1005C0003091200134FD1DC000932001C1E2D1E033
:1005D0001CC030914B0134FD14C000934B01CCE49E
:1005E000D1E013C0052710E000C000000BB91AC00D
:1005F000052710E0221F1DC010E021C04AE502C0FF
:1006000032ED432FC4E1D0E032E01AB114685F9AB2
:100610000BB11AB954E820E865E320FF05270BB9B0
:10062000279517951C3FF0F66695B8F7B1F720FFB0
:1006300005270BB9279517951C3FD0F627951795D9
:1006400017FF052700001C3F0BB9B0F629913A951A
:1006500019F70B7710913201110FC651D0400BB929
:1006600011F010932C0111E01CBB00681AB11B772C
:10067000402F4B7754E05A95F1F70BB91AB94BB9A3
:1006800069CFCF92DF92EF92FF920F931F93CF9398
:100690006B017C01142FC22F9695879577956795EE
:1006A00060587B47814E9F4FA70196010E9411051C
:1006B00069017A0181E0C81AD108E108F108809146
:1006C000C00082608093C0001092C100113021F1FF
:1006D00020E1129FA0011124C69528E0C29FC0010D
:1006E000112410E005501109000F111F802B842BDD
:1006F0008093C200C092C400D092C50088E180936C
:10070000C10087B98FEF88B9CF911F910F91FF90EA
:10071000EF90DF90CF90089540E350E0DDCFCF938E
:10072000DF938091C00085FF08C0E091E2028091D4
:10073000E1028E1711F0359903C02091E00226C026
:10074000F0E0E052FE4F80818093C6008091E2028B
:100750008F5F8093E2029091310197FFE2CF9091F9
:10076000E102891B81508930E0F210923101D9CF2A
:100770008217B1F09091C0003091C6009C7159F47D
:10078000F0E0E95AFE4F30838093DF01E091DF0112
:1007900081E08E0F8F779091C00097FDE9CF01C067
:1007A00044988091200184FF30C0C091DF01809186
:1007B000E002C81304C09091E302992331F1C81BF1
:1007C000CF77C93008F0C8E0DC2FD80FD7FF07C0BB
:1007D0009D2F9F77E7E5F1E0D0E0D91319C090E0B5
:1007E0006C2F895A9E4F0E94BB00D093E002CC230D
:1007F00049F0449AC83031F49091DF018091E002D1
:10080000981769F080E08093E302DF91CF9108951B
:100810002191DF01A158BF4F2C93DF5FDECF81E034
:10082000F2CF0F9360910D0170910E0180910F0135
:10083000909110010091110120911301409112013A
:100840000E9441031092E2021092DF011092E00236
:100850001092E1020F910895FC018381813049F4E7
:1008600088E690E09093300180932F01809168009A
:10087000089580EB90E09093300180932F0183E402
:100880000895FC0180818076803211F080E0089527
:10089000818190EE980F9230A8F0823261F48281CB
:1008A00080FD439A80FF439880911401811103C019
:1008B00082E080931401808187FDE8CF81E08093FE
:1008C000E302E4CF8FEF0895FC01ADE0B1E08C913D
:1008D000808311968C911197818312968C91129737
:1008E000828313968C9183838091130184838091FA
:1008F0001201858380911101868387E00895FC01B0
:10090000808180930D01818180930E01828180938B
:100910000F0183818093100184818093130195815D
:1009200090931201268120931101933010F01092C0
:100930001201813011F4109213010E94110481E020
:100940000895DC019091E202E091E102611108C09A
:1009500091509E1B993018F48FEF809331010895C8
:1009600081E08E0F891741F02C91F0E0E052FE4FAC
:1009700020838093E10211966150E6CF9EE088E1EA
:100980000FB6F894A895809360000FBE9093600016
:100990008BE78BB984E88AB9A8952FEF84E39CE0B4
:1009A000215080409040E1F700C000001AB880E874
:1009B00095E2A0E0B0E080930D0190930E01A0932A
:1009C0000F01B0931001109213011092120188E0F0
:1009D000809311010E9411040E94E60110921401FB
:1009E0001092E3027894A8950E94C3000E948F039E
:1009F000809114018823B9F390914B0194FFF3CFB8
:100A0000823059F468E082E091E00E94BF0080915A
:100A10001401815080931401E6CF62E08AE091E0F6
:100A2000F4CFA1E21A2EAA1BBB1BFD010DC0AA1F09
:100A3000BB1FEE1FFF1FA217B307E407F50720F047
:100A4000A21BB30BE40BF50B661F771F881F991FC2
:100A50001A9469F760957095809590959B01AC010B
:0A0A6000BD01CF010895F894FFCF07
:0C0A6A00FF5AA120000000000200030061
:00000001FF
